:0E20FD0000640005000100A00032000A00058A
:10163D00C10B4101250101A201011100410123004E
:10164D00C10AC1004100000041010100011A00C1A1
:10165D0003C182C108011700010A00011900C1016F
:101EEA00F583E0FCA3E0FDD39426EC940222C3ED33
:101EFA0094C8EC940022C2A1C2A5C2A2E509222577
:101F0A00E02494F8760008A60522F583E4F0A3F00D
:0F1F1A000524E5242225E02401F582E434002289
:10156800E4F5231212A19000007403F01220473012
:10157800092CC209900123E004F0E550D3940040FF
:101588000DD5500A1221497F0A7E0012212578576D
:10159800E6600B16E6B40106200503122065788B79
:1015A800E6D394034035E4F61221421213B2E4F56F
:1015B80018E51825E02495F9E7900126F06013E076
:1015C80014F0E0FFFDE518121F09EF7005AF1812BF
:1015D80020B80518E518C3940740D6E511609015A2
:1015E80011740B2511F8E614601414601A146023A2
:1015F800240370E7B204E4FDFF12200080DDE4FD5F
:101608007F0112200080D4122146E4FD7F021220BF
:101618000080C8200E04E51F70107B207DBC7C0074
:101628007F14121000751F078002151FE4FD7F0349
:0516380012200080A655
:1012A1007580FF759850758921758780758DFD75DD
:1012B1008BFD758A04758CF7D28ED28CD2A943BF6F
:1012C10002121E6AD2AFD2AC75090112139B7F5074
:1012D1007EC312212512139BE4F509F524E524129E
:1012E1001F1F121F14B480F5E4FDFC7F6312028CF2
:1012F100E49001F5F07B017A0179227F0D121F291B
:10130100EF70069001227480F07B017A0179257FCC
:101311000C121F29EF70087D01FC7F0C12028C90CA
:101321000125E0700E7D01FC7F0C12028C900125DD
:101331007401F07D0F7C007F0512028C7D167C000C
:101341007F0712028C7B017A0079007F08121F2926
:10135100E4FDFF122000E4FD7F02122000E4FD7F86
:1013610001122000E4FD7F03122000900125E064BA
:10137100027026FD7F04122000E4F524E52425E017
:101381002402F582E43401121F14B410EF9001F528
:09139100E030E703D20622C20697
:10139A00221221427F507EC31221251221427F5000
:0813AA007EC31221250221423D
:03000B00021D448F
:101D4400C0E0C0F0C083C082C0D075D000C000C065
:101D540001C002C003C004C005C006C007758A04E0
:101D6400758CF7788B06D20978A206E6D3940540E1
:101D7400027601121B5CD007D006D005D004D00334
:101D8400D002D001D000D0D0D082D083D0F0D0E027
:011D9400321C
:1020B800E511C39406500AAE110511740B2EF8A64B
:0220C8000722ED
:10200000ED701FEF25E024FDF582E43420F583E434
:1020100093FA740193FBEF25E02494F8A60208A636
:082020000322EDEF121F09225B
:10204700900000E0FF7006439B4075A303EFC39425
:0E205700014002D20AEFC394034002D20022DD
:0321460002148FF1
:1013B200900125E070183004055313FE8003431397
:1013C200013003055313FD8021431302801C3004B6
:1013D200055313FE8003431301E508D3940040072D
:1013E20015085313FD8003431302E4FFEF25E024A5
:1013F20031F582E43400121EEA5005121EF850083C
:10140200E512C313F5128008E512C3134480F512E6
:101412000FBF08D8E4FFEF25E02411F582E4340081
:10142200121EEA5005121EF85008E514C313F514F3
:101432008008E514C3134480F5140FBF08D8E4FFF5
:10144200EF121F1F121EEA5005121EF85008E51572
:10145200C313F5158008E515C3134480F5150FBFB6
:1014620008DEE4FFEF25E02421F582E43400121EB9
:10147200EA5005121EF85008E516C313F516800847
:0C148200E516C3134480F5160FBF08D810
:01148E00223B
:101B5C007580FF78A2E624FE601F14602E14603F8F
:101B6C0014605324047065C2A0121F006005E4F5D4
:101B7C00808003851280D2A622C2A6121F006005A7
:101B8C00E4F5808003851380D2A022C2A6C2A012E5
:101B9C001F026005E4F5808003851480D2A122C267
:101BAC00A6C2A0C2A1C2A2E5096005E4F58080032B
:101BBC00851580D2A522C2A6C2A0C2A1C2A5E509E4
:0D1BCC006005E4F5808003851680D2A2221A
:04214200759FA722BC
:0B212500EF1FAC0670011E4C70F6228C
:100C620000C1814001C0804101C0804100C181407A
:100C720001C0804100C1814000C1814001C080416A
:100C820001C0804100C1814000C1814001C080415A
:100C920000C1814001C0804101C0804100C181404A
:100CA20001C0804100C1814000C1814001C080413A
:100CB20000C1814001C0804101C0804100C181402A
:100CC20000C1814001C0804101C0804100C181401A
:100CD20001C0804100C1814000C1814001C080410A
:100CE20001C0804100C1814000C1814001C08041FA
:100CF20000C1814001C0804101C0804100C18140EA
:100D020000C1814001C0804101C0804100C18140D9
:100D120001C0804100C1814000C1814001C08041C9
:100D220000C1814001C0804101C0804100C18140B9
:100D320001C0804100C1814000C1814001C08041A9
:100D420001C0804100C1814000C1814001C0804199
:100D520000C1814001C0804101C0804100C1814089
:100D620000C0C101C30302C2C60607C705C5C40449
:100D7200CC0C0DCD0FCFCE0E0ACACB0BC90908C8B9
:100D8200D81819D91BDBDA1A1EDEDF1FDD1D1CDCA9
:100D920014D4D515D71716D6D21213D311D1D01019
:100DA200F03031F133F3F23236F6F737F53534F409
:100DB2003CFCFD3DFF3F3EFEFA3A3BFB39F9F83879
:100DC20028E8E929EB2B2AEAEE2E2FEF2DEDEC2C69
:100DD200E42425E527E7E62622E2E323E12120E0D9
:100DE200A06061A163A3A26266A6A767A56564A4C9
:100DF2006CACAD6DAF6F6EAEAA6A6BAB69A9A86839
:100E020078B8B979BB7B7ABABE7E7FBF7DBDBC7C28
:100E1200B47475B577B7B67672B2B373B17170B098
:100E22005090915193535292965657975595945488
:100E32009C5C5D9D5F9F9E5E5A9A9B5B99595898F8
:100E4200884849894B8B8A4A4E8E8F4F8D4D4C8CE8
:100E52004484854587474686824243834181804058
:03166D0001550024
:101AD1007E00E525252AFFEE3524FE22785BE6FE11
:101AE10008E67C00240022E52925E0FFE52833FEF5
:101AF10074012FF58274003EF583E524F0A3E525FA
:101B0100F022EF25E0FFEE33FE74392FF58274FFEA
:101B11003EF583E022E6F529F599C20C223EF52433
:101B2100D3E52594FFE5246480948022FFEC3ECF29
:101B3100249CF529EF34FFF528227854E6F599C263
:101B41000C227856E6F599C20C22C292E47855F639
:0B1B51007857F622785EE6FD7C00224B
:101E6A00121B4BFB7A0079517F067EEF122119E58E
:101E7A0051F46004E55170137B007A0079517F06B2
:101E8A00121F29EF700F7551FE800AE551FD7C0083
:101E9A007F0612028CE5516003B4FF037551FE22DE
:03214900021B4B2B
:0B213000C20CD2927F0A7E0002212523
:0300230002197B44
:10197B00C0E0C083C082C0D075D000C000C006C01C
:10198B000720980241117855E6C394325007E606BA
:10199B002459F8A699C2987855E6FFB401057550FD
:1019AB0032806AEF6407703A785AE6FE640360048B
:1019BB00EEB406089001F47408F08051EEB4100BED
:1019CB00200D089001F47408F08042EEB4100B78EF
:1019DB005FE624099001F4F080339001F47432F047
:1019EB00802B9001F4E0B5070B7550007857760605
:1019FB00D20D8019EFB40315785AE6B4190F900184
:101A0B00F47406F08007309904C299D20CD007D039
:0C1A1B0006D000D0D0D082D083D0E032C2
:10206500120601500F7508051221301207F71208E4
:0720750000120A5502214987
:10060100121ADDF527EC3EF5269001F4E0785566E7
:100611006002C3227859E6FFF4600AEF6551600574
:10062100EF6002C322785AE664197065FB7A00799B
:10063100597D04121DE68E248F25785D121ADFFF85
:10064100EC3EFEEF65257003EE65246002C322785F
:100651005CE6FF18E6FEC39F4004AD078002AD06CD
:10066100EEC39F4004AF068000E551C39D4006E5FF
:1006710051D39F4002C322788BE6FF7E00121E6099
:1006810012075CE529C39528500512076C80F4D345
:1006910022785AE6FF6403600CEF64066007EF649A
:1006A100106002C322785AE6FD64067039C3E5275B
:1006B1009408E5269400502E785CE6FFC39402501E
:1006C100099001F5E030E01EC322EFC39404500904
:1006D1009001F5E030E10FC322EFB408099001F574
:1006E100E030E202C322785BE6FE08E67A002400ED
:1006F100FFEA3EFEEF640A4E702AEDB4030E121EAD
:10070100297C007D05120EE27858A6057858E6642A
:10071100016002C32212075CE529C3952850051226
:10072100076C80F47B007A0079599001F4E024FE93
:10073100FD121DE68E248F259001F4E0FD2457F86B
:10074100E6FE74582DF8E67C002400FFEC3EFEEF37
:0A075100B52506EEB52402D322C33D
:10075B0022121E297C007D14120EE28D28E4F5294D
:0B076B00227F647E0012212505292258
:100A5500E4F52A785AE6FDB4061FE4F52A7459250B
:100A65002AF8E6F5997F327E0012212512214205EA
:100A75002AE52AC3940840E522ED6403600261A0DB
:100A8500121ADDF525EC3EF524785EE6F528785951
:100A9500121B16AF2912207C785AE6F529300CFD79
:100AA500120C12E52825E0F529300CFD120C12E593
:100AB5002AC395284002618F121AD1EF64634E70E4
:100AC50016F529300CFD120C1C9001F5E0F52930C6
:100AD5000CFD120C1C618B121AD1EF648C4E701038
:100AE500F529300CFD120C3C300CFD120C3C618BD1
:100AF500121AD1C3EF9464EE9400504AE52A2525D5
:100B0500FF7B007A007926121D95EF7004F526F516
:100B150027121AD1C3EF945AEE94004005E4F52943
:100B25008004E526F529300CFD120C26C3EF945AF6
:100B3500EE940040057529018004E527F529300C60
:100B4500FD120C46618B121AD1EF249CFDEE34FF89
:100B5500FCC3ED9480EC9400501A121B03F5293068
:100B65000CFD120C26121B03A3E0F529300CFD1217
:100B75000C468012E4F529300CFD120C587529013C
:100B8500300CFD120C58052A41B4300CFD121B3BEC
:100B9500300CFD121B43200C7380FB785AE6641061
:100BA5007027F52A7459252AF8121B16300CFD12E8
:100BB5000C50052AE52AC3940640E9121B3B300C6C
:100BC500FD121B43200C4580FB785AE66419703CE6
:100BD50018121B16300CFD120C50785A121B1630C9
:100BE5000CFDAF2912207C122142855129852999B6
:100BF500C20C300CFDAF2912207C122142121B3B86
:0C0C0500300CFD121B43300CFD1221428C
:100C110022852999C20CAF2902207C852999C20C11
:100C2100AF2902207C852999C20CAF2912207C7E34
:100C310000E525252AFFEE3524FE22852999C20CDF
:100C4100AF2902207C852999C20CAF2902207CAFF3
:100C51002912207C022142852999C20CAF29022048
:010C61007C16
:10080000752A01C210E4F52C785BE6FE08E6F97C57
:10081000002400FFEC3EFEF5288F29785AE6640696
:100820006002214DC3EF9464EE94004002210EE972
:1008300094015015785EE6FDE4FF120A4B7F011229
:100840000A374401120A1421B0785CE6D3940350AD
:1008500014121B557F02120A4B7F03120A374402FF
:10086000120A1421B0785CE66408702508121ADFB9
:10087000FDEC3EFC7F0812028C9001F5E04404F090
:10088000FD7C007F6312028C785EE6900000F02110
:10089000B0785CE6FF6405700221B0EF6407700277
:1008A00021B0EFB406091209FAF551D21021B0783F
:1008B0005CE6FFB40D091209FA900122F021B0782C
:1008C0005CE6FFB40C10120A07900125F0600221CB
:1008D000B075090121B0785CE6FFB41007120A0771
:1008E000F52A21B0785CE6B40A187858E66401600D
:1008F0000221B0121B557F0612028C785EE6F5517C
:1009000021B0785CE6FF121B5512028C21B0C3E5C2
:1009100029942CE5289401400221B0785BE67F0001
:10092000121AE0121B2DC3E5299420E528940050EB
:100930000AE529947FE52894005075785D121ADF46
:10094000F525EC121B1E5068121AE821B0785AE601
:100950006410705C785EE6F9785BE67F00121AE05E
:10096000121B2DE4FDE9FFC3ED9FEC9400504112F2
:100970002142E5292DFFE5283CFEC3EF9420EE94AB
:10098000005008EF947FEE9400501EED25E02460A7
:10099000F8E6FEED25E02461F8E67A002400F5256E
:1009A000EA121B1E5003121AE80DBD00010C80B59F
:1009B000E52A647F701B120A3F120A2A6003120A9A
:1009C0001D0526E526D3941040EFC2AF759F8080A9
:1009D000FEE52AB4FF07C2AF759F8080FE30101974
:1009E000122142120A3F120A2A6003120A1D05262A
:0909F000E526C3940B40EFC21090
:1009F90022785EE6FD7C0012028C785EE622785E43
:100A0900E6FD7C0012028C785EE622F0FD7C007F18
:100A19006302028CE42526FDE434EEFCAF270220B4
:100A2900927B007A007927AF26121F29EF22120242
:100A39008C9001F5E022752B77AF2B1220A5E4F5F8
:0C0A4900262212028C785DE6FD7C002263
:0907F700785676FF785476FF2253
:10207C007854E66FFF900C62937856667954F7EFBC
:05208C00900D6293F6C7
:01209100222C
:081DE6008B2A8A2B892C8D2D1C
:101DEE00752E00752FFF7DFFAF2D152DEF6026ABE5
:101DFE002A052CE52CAA2B7002052B14F9120E6263
:101E0E00652FFF900C62936D752E00F52FEF900DE0
:0A1E1E006293FD80D3E52FFEEDFF77
:011E28002297
:03167000014F0027
:101EAA00E52A25E02401F582E43400F58322E52AB7
:101EBA0025E024C1F582E43400F5832274D1252A71
:101ECA00F582E43401F58322C2B47F017E0022D276
:101EDA00B47F017E0022F0E52A24BCFDE433FC2213
:10148F00121F93E54F139290E54FA2E19291A2E2C2
:10149F0092937006C294D2958009E54FB41004D28E
:1014AF0094C295E54FC3940850077FB5121FE5808E
:1014BF0028E54FC3941050077FB1121FE5801AE53E
:1014CF004FC3941850077FB5121FE5800CE54FC32B
:1014DF00942050057FB1121FE5121FBCEF4E600321
:1014EF0002213B7F017E00122125120FC68E4D8FE8
:1014FF004E12155B8E248F2512155B8E268F2712A9
:10150F00213BE54E2525FFE54D35245403F5288F66
:10151F0029E54F7015E527B52925E526B528207D46
:10152F001FAF25AE241211578015E527B52910E5F9
:10153F0026B5280BE54F14FDAF25AE241211570524
:0B154F004FE54FD3941F4003E4F54F1D
:0E155A0022121F687F017E00122125020FC69B
:101F9300121ED2122125121F9F021F9FD2B5D2B447
:101FA3007F027E00122125C2B57F057E0012212506
:091FB300C2B47F027E0002212568
:101F6800E4FFFE20B50C0FBF00010EEF64644E7055
:101F7800F222D2B57F017E00122125D2B4C2B57FEC
:0A1F8800017E00122125D2B5C2B47B
:011F9200222C
:021FE500AD0746
:101FE7007B08ED3392B5121ED9122125121ED2128B
:081FF7002125ED25E0FDDBEAE8
:011FFF0022BF
:100FC600E4F52AF52BFD121ED9122125E52B25E085
:100FD600FFE52A33FEA2B5E433FBEEF52AEF4BF527
:0F0FE6002B121ED21221250DBD0ADBAE2AAF2B16
:010FF50022D9
:07213B00C2B5D2B4D2B522F7
:101FBC00E4F52AF52BFBFA20B50D121ED9122125BA
:101FCC00C2B47E007F00220BBB00010AEB64324AD4
:081FDC0070E5C2B47E007F0134
:011FE40022DA
:061157008D2AAB07AA0679
:10115D00121EAAE0FEA3E0FFC3EB9FFFEA9EFE1264
:10116D0020CAD3EF940AEE64809480400A121EAA1E
:10117D00EAF0A3EBF08028121EAAE0FCA3E0C39BCB
:10118D00EC9A5008121EC6E004F08013121EAAE05D
:10119D00FCA3E0D39BEC9A4006121EC6E014F0129D
:1011AD001EC6E0FBD3648094815008C3EB64809429
:1011BD007F5052D3EF9428EE6480948040127C00CF
:1011CD007D05120EE2121EAAEE8FF0120F1880305E
:1011DD00D3EB64809481400C121EAAE475F00112C9
:1011ED000F18801CC3EB6480947F5014121EAAE06C
:1011FD00FEA3E04E600A121EAA74FFF5F0120F183E
:10120D00121EC6E4F0121EAAE0FEA3E0D39400EE77
:10121D0094044009121EAA7404F0A3E4F0121EAA4D
:10122D00E0FEA3E0FFE4FCFD7B607AEAF9F8C3126F
:10123D000FB05007121EAAE4F0A3F0121EAAE0FE92
:10124D00A3E0FFC394C8EE94004009D3EF9426EEBB
:10125D0094024020121EB8E0FEA3E064024E6033FB
:10126D00121EB8E4F0A37402121EE07B027A007F16
:10127D0014021800121EB8E0FEA3E064014E6013C4
:10128D00121EB8E4F0A304121EE07B017A007F1455
:03129D0012180024
:0112A000222B
:1017D100E5432401FFE43542FEAD07FC2275F655D1
:1017E10075F6AA75F65543BF04228D828C83E49366
:0F17F10022AB42AA43A944227B007A007930221E
:0B2119008F828E83E493120E7B7F0107
:012124002298
:10209200AB071217DE8CF4AF058FF58BF675F78060
:0320A2007F00229A
:1020A500C2AF1217DEEF25E0F5F4E4F5F575F7821A
:0320B500D2AF2285
:061CF2008B4A8A4B894C6D
:101CF800120F2EFBAAF0530201EB24FFFFEA34FF78
:101D0800FE7C007D0F120E8DA905EB241DFFE43A21
:101D1800FEE97C00C3EF9DFFEE9CFED3EF94FFEE3F
:101D2800940140037F0022C3740F9DFFE49CAB4ADB
:0B1D3800AA4BA94C8FF0120F597F013D
:011D4300227D
:061C46008B448A4589462B
:101C4C00122142EF25E0F547754800854882F5835F
:101C5C00E493B433037F00220548E548700205473E
:101C6C00854882854783E493B4FF14AB44AA45A905
:101C7C0046E5478548F0120F911221427F01227BE5
:0F1C8C00007A007947121CF2EF70D5122142FF47
:011C9B002226
:0E210B00EF75F0148425E025412463020E7B5D
:0220ED00AC073E
:0E20EF00ED25E07B00FAAF04FC7D000220929C
:0A0FF600ED2401FDE43CFC02209212
:1020DC00AE07BE01037F0222BE02037F01227F00F6
:0120EC0022D1
:081BD9008F448B458A468947C1
:101BE100122142ED25E0F548754900854982F583CA
:101BF100E493B4FF037F00220549E54970020548DB
:101C0100854982854883E493FE740193FDEEB544D2
:101C110017ED6014AB45AA46A947E5488549F0127E
:101C21000F911221427F0122BEFF09BDFF06122141
:101C3100427F00227B007A007948121CF2EF70C0CB
:041C4100122142FF2B
:011C4500227C
:080776008B3D8A3E893F8D4056
:10077E00E4F543F544122142E54025E0FEE4240170
:10078E00FFE43EF5418F4285428285418374019399
:10079E00FEBE3314AB3DAA3EA93FE5418542F012A1
:1007AE000F911221427F0122BE770CE54445437022
:1007BE00068541438542447B007A007941121CF242
:1007CE00EF70C4E5444543700CAD40FF1220ED12AE
:1007DE0021427F0022AB3DAA3EA93FE5438544F06E
:0807EE00120F911221427F015C
:0107F60022E0
:0A18C4008E3D8F3E8B3F8A40894124
:1018CE008F828E837401937002FF22122142853E15
:1018DE0082853D83740293F5487F03E53E2403FD24
:1018EE00E4353DFCEFC3940F500E1217EBB4FF0816
:1018FE000F0DBD00010C80ECBF0F061221427F00C0
:10190E0022E54045416011853E82853D83E493ABDF
:10191E003FAA40A941120E7BE54345446038121799
:10192E00F2E4F5F0120F91E4F549E549C3954850FC
:10193E00251217F2120F2E75F000120F91ED254998
:10194E00F582E43CF583E493FF1217F2E48FF01274
:10195E000F59054980D4E5464547600BAB45AA466D
:0C196E00A947E548120E7B1221427F01C0
:01197A00224A
:0A1C9C008B358A368937AD07AC0698
:101CA6008D828C837401937002FF221221427F037E
:101CB600ED2403FDE43CFCEFC3940F500E1217EB2A
:101CC600B4FF080F0DBD00010C80ECBF0F061221FA
:101CD600427F0022E5364537600C1217EBAB35AA7A
:0B1CE60036A937120E7B1221427F014D
:011CF10022D0
:081D95008F2B8B2C8A2D892E67
:101D9D007532017B007A00792F853241AF2B1221EC
:101DAD000B7A0009AD2FAF2B121BD9EF601F852CBD
:101DBD0042852D43852E44754500754600754700B7
:101DCD007B007A007900AF31AE300218C40532E5E0
:081DDD0032D3940240BD7F00E7
:011DE50022DB
:081F29008F2D8B2E8A2F8930C9
:101F31007534017B007A007931853441AF2D12214E
:101F41000B7A0009AD31AF2D121BD9EF600DAB2E0D
:101F5100AA2FA930AF33AE32021C9C0534E534D32D
:061F6100940240CF7F0056
:011F67002257
:08170A008F3D8C3E8D3F8B40AA
:101712007B007A007942AD41121BD9EF601BAD43C9
:10172200AC42AF3FAE3E121A27EF700AAD43AC4255
:10173200FF120FF680037F01227B007A007942AF0D
:1017420041121C46EF701AE54125E0F5427543004F
:10175200FEAF43AD07FC7F331220921221427F007D
:1017620022AE42AF43AD07AC06AF3D122092E54038
:1017720075F002A4D3940CE5F064809480500A12B0
:1017820017D17F7712209280081217D17F3312204F
:1017920092E54324021217D5AF401220927901E953
:1017A200D395405024AF3FE53FE543240FFDE43598
:1017B20042FCE9FBC3ED9BFDEC9400FC122092E598
:0E17C2003EF53F753E000980D61221427F01A0
:0117D00022F6
:081A27008E448F458C468D476B
:101A2F0085464985474A854A82854983740193B41F
:101A3F0033037F00221221427402254AF54AE4350E
:101A4F0049F549854A82F583E493F548054AE54A05
:101A5F0070020549E4FD854A82854983E493B4FF0A
:101A6F0011EDD3940C500B054AE54A700205490D50
:101A7F0080E4E54875F002A4FFC3ED9FE5F06480B4
:101A8F00F87480985011E5472401FFE43546FEAD08
:101A9F0007FC7F331220927901E9D39548501DAF8F
:101AAF0045E545E9FDC3E54A9DFDE5499400FC1276
:101ABF002092E544F5457544000980DD1221427FEF
:011ACF000115
:011AD00022F3
:06028C008F2D8C2E8D2F3A
:10029200E4F53BF53CD3E52F94FFE52E94004005B1
:1002A20075380280037538017D011217F98D41AF4F
:1002B2002D12210BE53025E0F532753300853382AE
:1002C200F583E4937005AF301220A5853382853221
:1002D20083E493FFB4FF0874382DF8E4F6801274B7
:1002E200382DF8A605EFB477028D3CEFB433028DBA
:1002F2003B0DBD03B5122142E539701BE53A70177B
:10030200FB7A007930754101AF2D12210BAD307FA0
:10031200771220ED020564E5396006E53A60026174
:10032200D3E53C7006E53B700261D3E53C606412A4
:1003320017F9F541AF2D12210B7A007932AD30AFAA
:100342002D121BD9EF602812058760028142AD335E
:10035200AC32FF120FF6120564EF60028142120402
:100362004370028142120476700281420204B8850F
:100372003041AB38AD2FAC2EAF2D12170AEF600211
:100382008142120443700281421204767002814259
:100392000204B81217F91205726020120587600272
:1003A2008142AF3B1220DC8F41FB1204CF700281ED
:1003B20042120497700281420204FAAF3B1220DC1F
:1003C2008F417B001204CF6077120497607202049F
:1003D200FA7B007A007931853C41AF2D12210B7AEC
:1003E2000019120572602A1205E77054FB1205F417
:1003F20060121205E770491205326044120511605D
:100402003F02054D120532603712051160320205B6
:100412004D7B001205F4601BAD33AC32AF2FAE2E14
:10042200121A27EF701A1205B560151205946010A2
:100432000205D01205B5600812059460031205D0BA
:1004420022AF3C1220DC8F41FB7A007931AF2D12B2
:10045200210BAD317F771220ED853141AB38AD2FC5
:10046200AC2EAF2D12170A7B007A007932AD301212
:100472000776EF22754200754300754436754500D4
:100482007546007547357B007A007934AF33AE325A
:100492001218C4EF22754200754300754436754543
:1004A200007546007547357B007A007934AF33AE6C
:1004B200321218C4EF22853141AB35AD37AC36AFBD
:1004C2003412170AAD33AC32E4FF020FF67A007928
:1004D20031AF2D12210BAD317F771220ED853141E5
:1004E200AB38AD2FAC2EAF2D12170A7B007A0079F4
:1004F20032AD30120776EF22853141AB35AD37ACE4
:1005020036AF3412170AAD33AC32E4FF020FF67580
:1005120042007543007544367545007546007547BF
:10052200357B007A007934AF33AE321218C4EF2231
:10053200853141AB38AD2FAC2EAF2D12170A7B009F
:100542007A007932AD30120776EF22853141AB3530
:10055200AD37AC36AF3412170AAD33AC32E4FF021A
:100562000FF6853041AB38AD2FAC2EAF2D02170AF6
:10057200853B41AF2D12210B7A007932AD30AF2D80
:10058200121BD9EF22AD33AC32AF2FAE2E121A2787
:10059200EF22754200754300754436754500754675
:1005A200007547357B007A007934AF33AE321218CA
:1005B200C4EF22853141AB38AD2FAC2EAF2D1217CF
:1005C2000A7B007A007932AD30120776EF2285314C
:1005D20041AB35AD37AC36AF3412170AAD33AC325E
:1005E200E4FF020FF6AD33AC32AF2FAE2E121A2754
:0F05F200EF227A007932AD31AF2D121BD9EF22F3
:10167300011F076060016900000000000000000016
:101683000000000000000000000000000000000057
:101693000000000000000000000000000000000047
:1016A3000000000000000000000000000000000037
:1016B3000000000000000000000000000000000027
:1016C3000000000000000000000000000000000017
:1016D3000000000000000048012700000000000097
:1016E3000000480161FFFFFFFFFFFFFFFF4801C943
:0816F300FFFFFFFFFFFFFFFFF7
:10202800ED25E024C1F582E43400F583E022F58350
:0F203800EFF0FCF599C20C22F0FEF599C20C22D4
:0A1800008C2B8D2CA907AD03AC0260
:10180A00E52BF52DE52CFAECFBEDE4FF7F32785958
:10181A00E4F608DFFC7F32D2051221301207F7D234
:10182A000590012FE9122040AF0612207C9001306A
:10183A007406F0FE300CFD1218B2900131E52DF05D
:10184A00FE300CFD1218B2900132EAF0FE300CFDA7
:10185A001218BB900133EBF0FE300CFD1218BB904E
:10186A000134EDF0FE300CFD8E99C20CAF06122049
:10187A007C300CFD7854E6900135122040300CFD86
:10188A007856E6900136122040300CFD1221497F2D
:10189A00C47E09C20DC210200D0BEF4E6007EF1F68
:0718AA0070F51E80F2C2057B
:1018B100228E99C20CAF0602207C8E99C20CAF0613
:0318C10002207C86
:02100000AA073D
:10100200ECF524EDF525E4FD7D327859E4F608DDB2
:10101200FC7D32D2051221301207F790012FEA121D
:101022002039AF0412207C9001307410F0FC300C97
:10103200FD121133900131E524F0FC300CFD121148
:1010420033900132E525F0FC300CFD12113CE490A6
:101052000133F0FC300CFD12113C900134EBF0FC3A
:10106200300CFD121145EB25E0900135F0FC300CFF
:10107200FD121145E4FDEDC39B5037122028FEA35B
:10108200E0EEFA122028A3E0FE74362DF582E43455
:1010920001F583EAF0FC300CFD12114E74372DF588
:1010A20082E43401F583EEF0FC300CFD12114E0D9A
:1010B20080C4300CFD7854E6FF74362BF582E4349C
:1010C20001122036300CFD7856E6FF74372BF5827C
:1010D200E43401122036300CFD1221497F887E1340
:1010E200C20DC210200D0BEF4E6007EF1F70F51EF0
:1010F20080F2EF4E7004D210802B7B007A00795977
:101102007D06121DE6AB07AA06785FE6FE08E67CBE
:10111200002400FFEC3EFEEFB50308EEB50204C268
:10112200108002D210301004D20E8002C20EC2050C
:10113200228C99C20CAF0402207C8C99C20CAF04A1
:1011420002207C8C99C20CAF0402207C8C99C20CC8
:05115200AF0402207C47
:0E16FB004101F100015200C10F4201F2012C29
:0301000016000FD7
:03000000020200F9
:0C020000787FE4F6D8FD7581A202024769
:100E6200BB010689828A83E0225002E722BBFE028E
:090E7200E32289828A83E49322C1
:100E7B00BB010689828A83F0225002F722BBFE0156
:020E8B00F32250
:100E8D00BC000BBE0029EF8DF084FFADF022E4CC49
:100E9D00F875F008EF2FFFEE33FEEC33FCEE9DEC12
:100EAD00984005FCEE9DFE0FD5F0E9E4CEFD22ED58
:100EBD00F8F5F0EE8420D21CFEADF075F008EF2FA2
:100ECD00FFED33FD4007985006D5F0F222C398FD93
:050EDD000FD5F0EA2230
:100EE200C2D5EC30E709B2D5E4C39DFDE49CFCEE2B
:100EF20030E715B2D5E4C39FFFE49EFE120E8DC308
:100F0200E49DFDE49CFC8003120E8D30D507C3E402
:060F12009FFFE49EFE2299
:100F1800C5F0F8A3E028F0C5F0F8E5821582700264
:060F28001583E038F02201
:100F2E00BB010A89828A83E0F5F0A3E0225006878E
:100F3E00F009E71922BBFE07E3F5F009E319228950
:0B0F4E00828A83E493F5F07401932283
:100F5900BB010789828A83020F18500B09C5F02744
:100F6900F7C5F01937F722BBFE0D09F8E325F0F3B1
:100F7900C5F019E338F322F889828A83740193252D
:080F8900F0C5F0F8E4933822F2
:100F9100BB010A89828A83F0E5F0A3F0225006F7AB
:0F0FA10009A7F01922BBFE06F3E5F009F31922A8
:100FB000EB9FF5F0EA9E42F0E99D42F0EC6480C8B8
:060FC00064809845F02258
:101E2900AC1BAD1CAE1DAF1E780FEFA2E2EC20E695
:101E390001B35D5E5FF47004FCFDFEFFEF13FFEE7E
:101E490013FEED13FDEC13FCD8E08C1B8D1C8E1DCD
:101E59008F1EEE547FFE228E1B8F1CE4F51DF51E8E
:011E69002256
:1020CA00C3EE6480948040028007C3E49FFFE49ECD
:0220DA00FE22E4
:10020C00021568E493A3F8E493A34003F68001F28B
:10021C0008DFF48029E493A3F85407240CC8C333F3
:10022C00C4540F4420C8834004F456800146F6DFC2
:10023C00E4800B010204081020408090163DE47EFF
:10024C00019360BCA3FF543F30E509541FFEE493B7
:10025C00A360010ECF54C025E060A840B8E493A37E
:10026C00FAE493A3F8E493A3C8C582C8CAC583CAA9
:10027C00F0A3C8C582C8CAC583CADFE9DEE780BE61
:0117090000DF
:00000001FF
